:020000040000FA
:0200000048298D
:08000800F000030E8301F1007A
:100010000A08F2008A0183121F152308A20024088F
:10002000A3002508A4002608A5002708A600280884
:10003000A7002908A8002A08A9002B08AA002C0854
:10004000AB002D08AC002E08AD002F08AE00300824
:10005000AF003108B0003208B1003308B2003408F4
:10006000B3003508B4003608B5003708B6003808C4
:10007000B7003908B8003A08B9003B08BA003C0894
:10008000BB003D08BC003E08BD003F08BE00400864
:10009000BF001F1949281E08AC000319AC0A861BB3
:1000A0005228A20183161C08F8008312F81BA20133
:1000B0002208F7000A21F50A831272088A00710EDD
:1000C0008300F00E700E8B100B1609001430C10067
:1000D0008316981C69288312061A6C28030199005C
:1000E000C10B682808007D30C1008316981C762853
:1000F0008312061A792803019900C10B752808009C
:100100008316981C81288312061A84282208031952
:10011000220A99000800A101A0017320FF30A2006B
:100120008020A00AA01E8E28A001DB30A200802023
:10013000A00AA01E9528A001B730A2008020A00A26
:10014000A01E9C28A0019230A2008020A00AA01E20
:10015000A328A0016E30A2008020A00AA01EAA2819
:10016000A0014930A2008020A00AA01EB128A00151
:100170002430A2008020A00AA01EB828A0010130CF
:10018000A2008020A00AA01EBF28A0016620A10A0C
:10019000211F8E28A1010130A2008020A00AA01EEC
:1001A000CB28A0012430A2008020A00AA01ED228C3
:1001B000A0014930A2008020A00AA01ED928A001D9
:1001C0006E30A2008020A00AA01EE028A00192307C
:1001D000A2008020A00AA01EE728A001B730A2003C
:1001E0008020A00AA01EEE28A001DB30A200802003
:1001F000A00AA01EF528A001FF30A2008020A00ABE
:10020000A01EFC28A0016620A10A211FCB28A10165
:10021000A001080075084F3C031C15298313A0306A
:100220007507840077088000080075089F3C031C50
:1002300021298317D0307507840077088000831345
:1002400008008317F0307507840077088000831357
:10025000080076084F3C031C34298313A03076072E
:1002600084000008F700080076089F3C031C402922
:100270008317D030760784000008F7008313080046
:100280008317F030760784000008F7008313080016
:1002900083120313850186018316850123308500AF
:1002A0008601D130860027309B0036309C00C53057
:1002B0009D0040309F008312A9309F00981783163D
:1002C0000C309900181218151813981683128B17F2
:1002D0000B178316011783128B20F501F6010B16FD
:1002E000061A70298316981C7329831275087602E2
:0E02F00003197029292177089900F60A702950
:02400E00433F2E
:02401000FC3F73
:00000001FF
